S0160000755461736B657256312E345F424D2E7372656358
S10B8000F00B0020C5BC0000D8
S113801008B5034B03491868402201F01FFD08BD51
S1138020E8FCFF1F3CC0000008B5144B1880202852
S11380300ED004D800281CD008281DD119E08028AF
S113804017D080235B00984208D0402814D110E058
S113805061200B49062202F08FF80DE096210622DA
S11380606120C90002F088F8064B1A78064B1A7092
S113807002E0612002F0BAF808BDC046A0FDFF1F6F
S113808070170000E4FCFF1FCCFCFF1F37B5214D27
S113809021482968402202F00CFC00280FDA1C2039
S11380A02968402202F005FC0024A04209DA28686D
S11380B01A494022802401F0D1FCE40101E080242B
S11380C0240228680378212B04D01449402201F0AB
S11380D0C5FC0024124B29681868402201F0BEFC3C
S11380E080231B029C420CD169461C2007310122CB
S11380F002F0DFFB00280BDA022002F0F2FB00247E
S113810006E08023DB019C4202D1002000F058FAF3
S1138110201C3EBDE8FCFF1F1C8000003CC000008A
S1138120E0FCFF1F054B064A19781170FF22002856
S113813001D1044A12781A707047C046CCFCFF1F64
S1138140C0FCFF1FE4FCFF1F024B1A78024B1A709D
S11381507047C046C0FCFF1FCCFCFF1F1FB5011CAD
S1138160022368460372184B1B681A7BC272802272
S11381708280D200C280612202731A1C36321278C5
S113818042731A1C3732127882735B6800206A4685
S1138190009301F04BFB0D4C2070002810D00022FE
S11381A0052101F0A3FA009A520609D508490022D4
S11381B0207801F09BFA20788121002201F096FAC0
S11381C0207804B010BDC046E8FCFF1FE4FCFF1F8C
S11381D004040000F0B5554CA3B02568877B002D3E
S11381E04BD101F049FE019001F052FE061C281CFF
S11381F002F020FF402001F005FE4D4B18604020A6
S113820001F000FE4B4B1860281CFFF73FFF802352
S11382101B02984201D00123236000F099FB6D20DA
S1138220042101F073FF0320FFF798FF00287BD09F
S1138230414B42481A78424B1A7001F063FD4148A1
S113824001F060FD019B0A219E1BB0B201F06BFDA1
S11382503D4801F057FD01F00FFE8A2101F063FD56
S11382600BE06B46D87A1A7B00280ED1D2B2062ACC
S11382700ED0832A01D103F0E7FC381C02A90522A1
S113828001F04CFA0028ECD11FE0012807D016E0D9
S1138290294B2E491878162201F012FDEDE7D2B2CF
S11382A0B72A06D0DD2AE8D12368082BE5D120605F
S11382B0E3E703F0A7FC264801F024FDDDE792B2D2
S11382C0381C02A901F02AFAD7E7226837231A4298
S11382D02AD0194D287801F031FA002824D02878C2
S11382E002A9402201F01AFA041E1DD002A8211C82
S11382F000F02AF9174B02A81A88211C002A0FD172
S113830001F0B0F80028EAD08020400000F0EAF93B
S11383100228E4D128781049172201F0D1FCDEE7C5
S1138320002201F09FF8DAE723B0F0BDECFCFF1F58
S1138330E8FCFF1FE0FCFF1FE4FCFF1F7CC0000003
S1138340CCFCFF1F99C00000A8C00000D8C00000EA
S1138350AFC00000A0FDFF1FC1C000007047021C99
S11383600878131C002806D01B780131013298428A
S1138370F6D000200AE000229A56202A06DC0022C9
S11383809A56202A01D10133F9E7181C704730B5F9
S11383900368021C00215956202904D111680133B5
S11383A001311160F6E71D1D0020AB4216D019788B
S11383B04CB22F2C12DDCCB2211C30390001C9B2D1
S11383C080B20133092902D9211C3739C9B20F24DB
S11383D021400843116801311160E6E730BD0368AC
S11383E000229A56202A05D01A7820218A4301D0E7
S11383F00133F9E700229A56202A01D10133F9E723
S113840003600020185643425841704708B5054898
S113841001F078FC044801F075FC044801F072FC9A
S113842008BDC04668C2000059D000007BC20000ED
S1138430F0B52C4A2C4E13780C2253439C59F31854
S11384401A798BB0071C019203A820211B225D79A5
S113845001F0FCFA002F04D0BD4225DD0C34013DAF
S1138460FAE7224801F04EFC1E4A13780C225343CB
S1138470F618B06801F046FC1D4801F043FC13E017
S1138480206801F03FFC019B021C30789A421EDBFD
S113849003A9012201F014FC606801F033FC1548C3
S11384A001F030FC0C34013D002D15D0124E00219A
S11384B03078422201F004FC0028E1D130784021D8
S11384C00E4A01F013F90E4B01201D6007E0019BD9
S11384D003A99A1A92B2DDE7094B281C1D600BB060
S11384E0F0BDC046A8FDFF1FA0CD00007AC2000069
S11384F07EC200007BC20000CCFCFF1F6D10000098
S1138500F8FCFF1F10B5847B88B0201C6946052247
S113851001F004F9002813D06946CB780A79012BBD
S113852008D1DD2AF1D1074B18680028EDD0FFF7F8
S11385307FFFEAE792B2201C694601F0EFF8E4E716
S113854008B010BDF8FCFF1F08B50A1C0349031C42
S11385500878191C01F0B4FB08BDC046E4FCFF1FF9
S1138560154B164A1B6812685868516810B50124E7
S1138570884208D1D88ED18E884204D1117B1C7BCD
S1138580641A611E8C4152895B895340282213422C
S113859001D0022214430422134200D01443DA0609
S11385A001D508231C430120FFF770FDE30702D522
S11385B00420FFF7D3FD10BDE8FCFF1FE0FCFF1F04
S11385C038B50A4C051C21680948402202F050F9CC
S11385D0012D08D0022002F084F9064B21681868A6
S11385E0402201F03BFA002038BDC046E8FCFF1FE2
S11385F01C800000E0FCFF1F08B5044B021C1B6834
S1138600C021D86B01F02CF908BDC046E8FCFF1F5F
S11386107FB5054801F076FB01A8FFF7EDFF01A83F
S113862001F070FB07B000BD96C200007FB5031CCB
S113863002380B2845D803F03DFC06441144444459
S11386403A351825182DFFF7E3FFFFF7DFFE1E4824
S113865001F058FB1D4B1868213020E01B4B1422FD
S11386601868213001F0FAF92BE00C3B581E8341C5
S11386700420C01A01A902F03FFB01A801F042FB4B
S113868013480CE0102002F037FB124801F03AFBCB
S11386900C2013E01020002102F02EFB0E4801F004
S11386A031FB0EE0082002F027FB0C4803E02020F9
S11386B002F022FB0A4801F025FB0A200021FFF703
S11386C0B5FF07B000BDC046A8C20000E8FCFF1F0C
S11386D045C40000C0C20000D0C20000E0C20000D7
S11386E0EFC20000802310B55B0098420BD1164BFB
S11386F002241B88002B25D1144B1B88002B21D16D
S1138700FFF792FC03E08022104B92001A80104B7A
S11387101A8880235B009A4202D12020FFF784FC50
S1138720FFF776FFFFF772FE0A4801F0EBFA0A4BF7
S113873000241868213001F0E5FA084B201C1C7055
S1138740FFF776FE201C10BD9EFDFF1FF6FCFF1FE9
S1138750A0FDFF1FA8C20000E8FCFF1FA8FDFF1F2B
S113876032280FD0332819D0312824D1134B144A7E
S1138770186812681968134B10401B688B43184320
S1138780800116E00D4B0E4A1868126819680D4BEB
S113879010401B688B431843C0010AE0074B084A8A
S11387A0186812681968074B10401B688B431843FC
S11387B00006C00F00E000207047C04654F00F4090
S11387C040F00F4050F00F40F7B5134F01253B68C0
S11387D031201A1C38321278002400925B8F0193E6
S11387E0461C40B2F6B2FFF7BBFF002800D02C4372
S11387F06D00EDB2392E01D0F0B2F1E7FFF7B0FE13
S11388003B6800991A1C383211705470019A002088
S11388105A87FFF7D5FEF7BDE8FCFF1F322807D0C3
S1138820332809D031280DD1074B1B685B0E06E0B5
S1138830054B1B681B0E02E0034B1B68DB09012080
S1138840984300E00020704754F00F4038B5031CF3
S1138850303B0020032B4BD8181C03F02BFB0209E0
S113886005078024A40405E0802403E0002401E03B
S1138870802464045DB264290BD003DC00206129E8
S113888036D003E0692904D06F291AD00120404270
S11388902EE0184BE2431968012011401960164B71
S11388A019680A401A60211C021C03F0E7F8134BF4
S11388B01A680123AB4038321D1C1378AB43137084
S11388C015E00C4B211C1A680120A2431A600022F7
S11388D003F0D4F8084B1A6814431C60074B1A6859
S11388E0012338321178AB401D1C0D431570002054
S11388F038BDC04658F00F4054F00F40E8FCFF1F4D
S1138900104BC10704D51968802292040A4302E07F
S113891019680D4A0A401A601968820703D5802233
S113892052040A4301E0094A0A401A6080224107BE
S113893002D519680A4302E0196891430A1C1A60B7
S11389407047C046400000F8FFFFFFFDFFFFFFFE39
S11389500F4B70B51B6801211A1C38323933167855
S11389601878012430401870FFF7CAFF30206921BD
S1138970264200D06F21451C49B240B26400EDB2DA
S1138980FFF764FFE4B2382D01D0281CEFE770BD77
S1138990E8FCFF1F1E4B10B51A68041C110619D4FD
S11389A01A68910718D41A68510717D41A689106DF
S11389B016D41A68510615D41A68910514D41A6885
S11389C0510513D41A68110512D41B689A0411D5E1
S11389D0104910E010490EE010490CE010490AE07B
S11389E0104908E0104906E0104904E0104902E08B
S11389F0104900E01049002C04D1081C01F082F950
S1138A00201C04E0201C01F0C1F9001BC0B210BD01
S1138A10008004408CCD00004CD0000080CE0000CB
S1138A2044C2000064C100002BD00000EFC000006D
S1138A30A8C1000024CE000032CE000038B503F0F7
S1138A40CDF80024051C012C03D0022C03D00948C6
S1138A5002E0094800E0094801F054F9A54202D1B6
S1138A60074801F04FF90748013401F04BF9032C92
S1138A70E9D138BDFEC2000006C300000FC30000E8
S1138A8018C3000045C40000F0B50C1C93B0161CBC
S1138A90072801D900F0A3FC03F016FA08003900F6
S1138AA0B102CE02A1042C0388048D04081E05D053
S1138AB0042908D10122BD4B00201A70FFF7B8FC2D
S1138AC0051C00F09DFC02220529F4D0032206298E
S1138AD0F1D004220729EED005220929EBD0062281
S1138AE00A29E8D007220E29E5D008220F29E2D06E
S1138AF009221029DFD00A221129DCD000251229ED
S1138B0001D000F07DFCA94B281C1D70D6E706920D
S1138B10272901D900F063FC081C03F0D5F92800CB
S1138B204000D5006004C300890060046004600450
S1138B3060046A007500C00060046004EC00DC019D
S1138B40DC01600460046004600460046004600488
S1138B5060046004600460046004600460042C0029
S1138B60EC00DC01DC01600452023400380003F044
S1138B706BF800F034FC8E4801F0C4F80020FFF7D5
S1138B8009FF00F02CFCFFF759FF00F028FC101C33
S1138B9000F039FFC0B203F035F800F020FC85483E
S1138BA001F0B0F8844801F0ADF8844801F0AAF867
S1138BB001F06EF90A2101F0B6F8814801F0A2F83B
S1138BC001F05AF90A2101F0AEF808AC7D4801F031
S1138BD099F8201C01F03AF90A2101F0A4F87A4826
S1138BE001F090F820880A2101F09DF8774800F000
S1138BF0F4FB08A802F04EFA00250570744801F051
S1138C0081F808A800F0EDFB1378313B032B01D960
S1138C107048E2E3704801F075F8069900200856A0
S1138C20FFF7FCFD051E01D16C48DAE36C48D4E380
S1138C301078031C313B032B01D96A48CDE340B2C1
S1138C40FFF7ECFD051E01D06748C6E3041C0126AE
S1138C503120471C40B2FFB2FFF782FD002801D04B
S1138C603443E4B27600F6B2352F01D0F8B2F0E71F
S1138C70069800F0ACFEC6B20698013E0123B3404C
S1138C8001301E1C069000F0A2FE012801D13443DD
S1138C9000E0B443E0B20021FFF732FEB0E3FFF797
S1138CA093FD9CE31378313B032BC6D84F4801F066
S1138CB029F8069A00201056FFF752FD051E01D030
S1138CC04B488AE34B488CE3101C079200F07FFE6C
S1138CD0041C07A8FFF783FB002801D046487CE367
S1138CE0079B2F34002160B25956FFF7AFFD0028CF
S1138CF000D174E3F2E70023D356002B02D11021F4
S1138D00029127E0101C00F062FE3C4B186006A89C
S1138D10FFF765FB069B1A78002AF0D020218A43CE
S1138D2052B204214C2A02D0572A04D10221344AD7
S1138D300133116005E0422A04D1314A0121116056
S1138D405B18069306980023C356002BD7D000F077
S1138D505AFE02902B4800F0D5FF08AB20221A706F
S1138D605A70029B002B00DC39E3244D0C21286847
S1138D7000F0D9FF244800F0C5FF6A4622321023D0
S1138D80009203931E4E3268022A45D0042A56D01C
S1138D90012A00D023E3212C38D16F4616372868E6
S1138DA0391C02F0E9FC3B7832E0C046A8FDFF1F05
S1138DB022C3000036C3000081C200004DC300007E
S1138DC0A8C000005AC300006CC300006FC30000B9
S1138DD073C3000098C30000AAC30000BDC3000011
S1138DE0C6C30000CEC30000DDC30000EDC3000015
S1138DF0FAC30000FEC3000002C40000A4FDFF1F6C
S1138E00C8FCFF1F0AC400001BC4000029680B78BB
S1138E100793079AD0B20EE0212C07D16F4616377C
S1138E202868391C02F0A8FC3B8801E029680B88FB
S1138E300793079A90B23378202119430DE0212C2F
S1138E4004D1286807A902F097FC02E02B681B688C
S1138E500793337820210798194300F064FF2968A9
S1138E6033685A182A60039A0799D21A0392019117
S1138E70022B06D0191F48424141182249420A4098
S1138E8000E00822009FF9188C4667450CD0019831
S1138E902E21D040061C203EF6B25A2E00D8C1B274
S1138EA03970083A0137F0E7009AD218029B009211
S1138EB0013B0293002B03D00399002900D061E702
S1138EC0009A0D2313700A2353700023937008A88B
S1138ED000F018FF45E70023D356002B00D17EE2B3
S1138EE0101C00F074FD051C112C01D0232C01D1A1
S1138EF0B24800E0B24800F005FF06A8FFF76FFA99
S1138F00069B1A78002A00D169E220218A4352B2D2
S1138F1004214C2A02D0572A04D10221A94A013340
S1138F20116005E0422A04D1A64A012111605B18B0
S1138F30069306A8FFF753FA069800F048FD089038
S1138F4006A8FFF74CFA112C02D00123232C08D1D8
S1138F500698002282560123002A02D000F053FD15
S1138F60031C223CE4B200260122A24276411C1CCE
S1138F70002C00DC33E2934F3A68022A0BD0042A17
S1138F8014D0012A19D1089B002E02D007A90B7016
S1138F9006E02B7011E0089B002E05D007A90B807A
S1138FA0281C02F09FFB08E02B8006E0002E02D074
S1138FB0281C08A9F5E7089929603B68013CED18CD
S1138FC0D6E70023D356002B00D108E2101C00F092
S1138FD0FEFC041C06A8FFF702FA0698002282563B
S1138FE000218A4202D000F0F2FC011C201C02F095
S1138FF05FFB051E01D17448F3E17448EDE10029DB
S113900009D0032900D0EAE1714B101C1C6800F060
S1139010FAFC2081E3E16F4D2B88042B05D16E48C7
S113902000F070FE10232B8004E06C4B081C1980A8
S1139030FEF7FAFF251CE3E10892072900D9CEE1E7
S1139040081C02F037FF04244148134D523808A885
S1139050FFF79DF9041C08A8FFF799F907A9087000
S11390600122201C01F004FC5D48B6E108A8FFF7CA
S11390708EF9041C08A8FFF78AF907A90870594853
S113908001220443A0B201F0F3FB5748A5E108A86C
S113909007ACFFF77CF9211C012201F00AFC00282F
S11390A007DB524800F02EFE2078812100F03BFEC1
S11390B095E14F4891E1464B402218684D4B1968A1
S11390C000F0CCFC4C4888E1FEF7A2FF0020FFF73B
S11390D077FA4A4881E1012001F003FC48487CE129
S11390E0022001F0FEFB474877E10020FFF768FA11
S11390F0454872E1162900D971E1081C02F0E4FE2A
S1139100170090002A004000AE006F016F016F014C
S11391106F016F016F016F016F016F016F016F01CB
S11391206F01CC006F016F016F013F013F01284BBC
S113913000241D6807206043344B311C181800F0CC
S11391400CFE002801D12C732CE101340C2CF1D13C
S11391502F4842E10023D356372B05D11C4B012263
S11391601B6859680A4307E0382B07D1184B0122C2
S11391701B68596891430A1C5A6013E125482CE185
S1139180134B00241D6805206043234B311C181821
S113919000F0E3FD00280CD16A6806239A43131CEF
S11391A0002C04D0012C00D015E102224FE004224F
S11391B04DE00134032CE6D118480EE120C4000030
S11391C027C40000C4FCFF1F2FC4000038C40000E3
S11391D0E8FCFF1FF6FCFF1F48C400009EFDFF1FB4
S11391E054C400000080FFFF66C400007EC4000079
S11391F093C40000E0FCFF1FB5C40000D6C4000007
S1139200F6C4000011C500002EC5000010C1000006
S1139210EEC5000046C500001CD0000007C60000D3
S1139220794B00241D687948A300C018311C00F054
S113923094FD00280DD16968182399430B1C012C57
S113924004D0022C00D0C6E0102200E00822134310
S1139250C1E00134032CE6D16D48BEE06A4B002422
S11392601F686C48E300C018311C00F076FD051E31
S11392700DD07A6860239A43131C012C03D0022C6E
S113928003D1202200E0402213437B608AE00134B2
S1139290032CE6D16048A4E0604800F033FD604848
S11392A000F030FD584C21680B7B0B2B04D80720B1
S11392B043435C48C01800E05B4800F023FD5B4D6D
S11392C0281C00F01FFD23682E1C5B68DA0701D5FB
S11392D0574800E0574800F015FD574800F012FDCC
S11392E023685A680123910704D404231A40534283
S11392F053415B00052043435048C01800F002FD71
S11393004F4800F0FFFC236802205B68DA0601D4B2
S11393101807C00F3D4B8000181800F0F3FC4948B3
S113932000F0F0FC236801255B68590602D49D0611
S1139330ED0F6D00444800F0E5FC3648EB00C01822
S113934000F0E0FC301C00F0DDFC002D47D03F486D
S113935000F0D8FC236800213633187800F0DAFCDA
S11393603B4D281C00F0CEFC3A4800F0CBFC2368AF
S113937000213733187800F0CDFC281C2DE0101C98
S113938000F041FBC0B2632803D8002802D10120B9
S113939000E063201C4B1B68152C01D1363300E020
S11393A0373318700420FEF7D9FE18E0081C111C8E
S11393B0FFF73CF913E0062911D12748111C00F0EE
S11393C0CCFC051E16D02548311C00F0C6FC051E39
S11393D00AD0234801E06B60E4E700F093FC002529
S11393E00EE000F08FFC0BE0074B40211B685A890C
S11393F08A4304E0044B40211B685A890A435A817A
S1139400281C13B0F0BDC046E8FCFF1F36CE000098
S11394101AC6000034D0000030C600005EC500004B
S113942077C5000010C100007FC5000045C40000DE
S113943088C500008AC500008CC500001CD000004F
S113944010C6000094C50000A3C50000B1C500000B
S1139450BDC50000C1C50000CCC50000D3C50000D7
S1139460DBC50000F0B585B003910021071C029212
S113947001910399002900D1F8E03B787D4C082B39
S11394800CD17D4B1A78002A05D07C48013A013072
S11394901A7000F037FC00232370E2E01B2B04D089
S11394A05B2B05D122781B2A02D123700137D8E027
S11394B022785B2A4BD1181C4138032847D802F084
S11394C0F9FC101009026C4B1A78002A00D1C8E08C
S11394D0013AC5E0684B1A78272A00D9C1E0013265
S11394E0BEE0674C28202268664E5043301800F0D6
S11394F059FC3B78051C412B08D12368002B01D172
S1139500032300E0013B23605F4806E02368013346
S1139510032B00DD00235D48236000F0F3FB002DE6
S113952004D05B4800F0EEFB013DF8E7574800F03B
S1139530E9FB206828256843301800F0E3FB206825
S11395404543701900F02EFC4B4B187089E00A2B30
S113955000D186E0002B00D183E04749484C0A78CB
S1139560216828256943474E89188B553B780D2B74
S11395706AD10A2302988B55FEF7D4FD23683E4A2C
S11395805D431378434A0C20127843494243013324
S113959075195458DBB28A185679EA180021013A31
S11395A011700299002905D13C4A1288002A39D049
S11395B0510537D4002B32D0281C002E19D0216835
S11395C0FEF7CDFE013E0190002810D0344800F093
S11395D099FB207A617A019AFFF756FA002802D1A2
S11395E0304800F08FFB029A002A1BD112E00C34A1
S11395F0E2E72D49FEF7B3FE021E10D00420092134
S1139600FFF742FA002802D1264800F07BFB029BB8
S1139610002B07D1214B1888FEF706FD02E02348F2
S113962000F070FBFEF790FD134B00221A70144BF0
S113963019680131032903DC19600121019106E055
S11396401A600122019202E00B4B01321A70094B9D
S113965000221A70084B01371A78272A01D92722C9
S11396601A70039B013B9BB2039302E7019805B078
S1139670F0BDC046F4FCFF1F9CFDFF1F55D0000049
S1139680F0FCFF1FFCFCFF1F49C600007CC2000069
S11396901EC40000A8FDFF1FA0CD0000A0FDFF1FF9
S11396A045C4000006C400004DC6000002C400000A
S11396B013B5441EE4B21423634304480068C3187A
S11396C0187C00945C680323A04716BDACFDFF1F03
S11396D008B5044B18701423584300F093FB024B55
S11396E0186008BDA9FDFF1FACFDFF1F37B5031CA3
S11396F00D1C0020FF2B0DD0013BDBB214245C4376
S1139700054909680C19207C0093111C64682A1C03
S11397100223A0473EBDC046ACFDFF1F13B5441E47
S1139720E4B21423634304480068C318187C00940B
S11397305C680423A04716BDACFDFF1F421ED2B2D5
S1139740142313B5534305490968CB18187C002129
S113975000925C680A1C0523A04716BDACFDFF1FE0
S113976030B50A4B0A4A1B6814780022A2420BD077
S11397705D680132854204D11D7C8D4201D1D0B295
S113978003E0D2B21433F1E7002030BDACFDFF1F7B
S1139790A9FDFF1FF0B5061C85B0101C01910292B3
S11397A00393FFF7DDFF011E01D000203AE0FFF72D
S11397B0D7FF071EF9D0142545431B4B143D1B68E6
S11397C05D193388002B13D0039800F01BFB041C95
S11397D0A8600DD03388181C009300F013FB0028F8
S11397E0E3D0009B20606060A060C018E060E3826A
S11397F07388002B11D0039800F004FB041CE8606C
S11398000BD07688301C00F0FDFA0028CDD0206003
S11398106060A0608019E060E682029B381C6B6087
S1139820019B2B7405B0F0BDACFDFF1F07B50028EC
S11398300ED0002103280FD1108901AB12681880C3
S113984059801178181C054A1823FFF7A3FF04E078
S1139850101C00F0BFFE00E0081C0EBDE19A0000E1
S11398602023F7B50E1C141C194203D013700823CF
S11398709E430134730706D5002804DA2D23237090
S11398804742013400E0071C00232E4D0093002FB3
S113989036D0BD4213D9281C0A2102F01FFB009BBD
S11398A0051C002B03D10128F3D1730601D5302305
S11398B002E03307EDD5202323700134E9E7002DBE
S11398C001D001230093291C381C02F007FB631C00
S11398D00193031CC0B26843303323703F1A0A213A
S11398E0281C02F0FBFA019C051CD0E7002B0DD0CC
S11398F0281C0A2102F0F2FA30232370051C0134DB
S1139900201C009B002DF1D1002B0DD1330703D572
S11399102023601C237007E0730602D53023601CEB
S1139920237030230370013073B2002B04DA0D234B
S113993003700A234370023010231E4000D10670C6
S1139940FEBDC04600CA9A3BF7B5202300901942D9
S113995001D013700132080704D530231370782323
S11399605370023240230B409C46CBB21026019325
S113997007230E4019400F1C042900D904277F0037
S1139980FFB2141C3B1C013BDBB2FF2B11D000982F
S11399909D00E8400F21051C0D40291C3031392958
S11399A004D960462731002800D0203921700134C1
S11399B0E9E70199D0194BB2002B04DA0D230370A7
S11399C00A2343700230002E00D10670FEBD10B58C
S11399D0031C00229A56202A01D10133F9E7002002
S11399E01A7851B22F290DDDD2B20101101C303882
S11399F0C0B20133092803D9101C57380F24204062
S1139A000843EDE710BD10B500220378191C303966
S1139A10092906D9002B17D02D2B00D101220130A2
S1139A20F3E7002301780C1C303C092C07D85C00B8
S1139A30303CDB00E31849B201305B18F2E7181C34
S1139A40002A02D0584200E0181C10BD031C8218E2
S1139A50934202D019700133FAE7704710B500231E
S1139A60934203D0CC5CC4540133F9E710BDF7B57D
S1139A70038A041C0E1C4768151C9A4200D91D1C3D
S1139A80ADB2002D28D0E3687A1962609A4215D3EA
S1139A90DB1B9BB22268E91A00935318636001919F
S1139AA001F04AFC002E12D0391C009A301CFFF73A
S1139AB0D5FF009B2168F018019A06E001F03CFCF8
S1139AC0002E04D0301C391C2A1CFFF7C7FF01F0FC
S1139AD02BFC238A5B1B238201F02EFC281CFEBD79
S1139AE0F7B51D1C08AB1B78171C14225A43164EDD
S1139AF00191316800928B189C6801F015FC052DCA
S1139B0009D0062D09D0042D16D1201C01993A1C28
S1139B10FFF7ADFF16E0258A11E0012F03D133686A
S1139B20009A9B18DC68002C08D02368258AA3605F
S1139B3063600023238202E0002500E0251C01F07D
S1139B40FBFB281CFEBDC046ACFDFF1FF7B5041C83
S1139B50151C0F1C01F0E8FB218A628AE38A88182D
S1139B604019984202DD5D1AAD1AADB2A168AA1877
S1139B70628201914A19E168A2602E1C8A4205D3CF
S1139B80D31A2268A3609B1AEE1AB6B201F0D4FB72
S1139B900198391C321CFFF761FFB54204D0B91992
S1139BA0AA1B2068FFF75AFF01F0BEFB638AA28A52
S1139BB0AB4206D1238AEB189A1800232282A3828F
S1139BC002E0AA18A2825B1B638201F0B5FB281C89
S1139BD0FEBD0000F7B5041C0191002936D10278BE
S1139BE043780D1C9A4261D101F09EFBA178304B61
S1139BF030481970FFF7B4FD2F49087000280ED0C3
S1139C00142250432D4B1B6818181438836820798C
S1139C101A8A561D3618D88A864203DD0D7001F063
S1139C208BFB43E006321A82A11D8C420CD09A6849
S1139C30501C9860207810709868DA68904201D3BC
S1139C40186898600134F0E706252FE01A4B1E7857
S1139C50002E0DD102784378351C9A4226D187789C
S1139C601448391CFFF77CFDFFB2061E06D11DE027
S1139C700F4A177800221A7001F05EFB14220F4B72
S1139C8056431B689E19E378143EB068032B04D135
S1139C90C58A038AED1AADB208E0211C019AFFF7C8
S1139CA055FF0421051C78B200F030FA281CFEBDD3
S1139CB0ABFDFF1FE19A0000AAFDFF1FACFDFF1FD3
S1139CC008B5031E04D1081C111CFFF783FF05E02F
S1139CD00020FF2B02D0181CFFF7EAFC08BD38B5A2
S1139CE0041C031C1A1B0133581E057892B2002D64
S1139CF0F8D1281C002A03D0081C211CFFF7E0FF20
S1139D0038BD000008B5024B1978FFF7E8FF08BD1D
S1139D10CCFCFF1F1FB56A46FFF7A2FD6846FFF79C
S1139D20F1FF05B000BD1FB56A46FFF70DFE68469A
S1139D30FFF7E8FF05B000BD07B5031C0020834210
S1139D400AD06A46107050709370117101236846EE
S1139D500521D370FFF73EFF0EBD0378002B0FD013
S1139D6000228A565BB2934207D0D80FD1179A4289
S1139D70484140420123184307E001300131ECE738
S1139D8000200856431E98414042704710B5031CFA
S1139D900C78181C1C700A78013352B20131002A65
S1139DA0F6D110BD021C031C981A0133591E097800
S1139DB049B20029F8D170470E4B13B500221A801E
S1139DC00D4B0E4A19600E4B147819601A1C037857
S1139DD0A34203D0002B0CD00430F8E74388C91801
S1139DE011606B460733994203D855230B70013138
S1139DF0F7E713BDB4FDFF1FB0FDFF1FD2FCFF1F2B
S1139E00B8FDFF1FF8B50E4F0E4E3B683488051C95
S1139E101C1903231C4201D09C4304340A4A6319CD
S1139E2012689A420AD92A1C201C0021FFF70EFE50
S1139E303B68201CE31AED18358000E00020F8BDD3
S1139E40B0FDFF1FB4FDFF1FB8FDFF1F094B10B588
S1139E501A68011C131C981A01331C7880B2552C03
S1139E60F9D0002800D11A1CBF231B019A1A0A80BA
S1139E7010BDC046B8FDFF1F034B1868034B1B6899
S1139E80C01A80B27047C046B8FDFF1FB0FDFF1F67
S1139E90044B1868044B1B68C01A044B1B88C01A77
S1139EA080B27047B8FDFF1FB0FDFF1FB4FDFF1F58
S1139EB0F0B585B00392564F564A002313603B60B9
S1139EC0554B02901B780C1C2678002E44D09E42E1
S1139ED03BD1231CE51A00260134A657EDB2002E0F
S1139EE0F8D1142068430430FFF78CFFEB43E318E8
S1139EF038600193371C019C6278002A23D0029BAE
S1139F00196800291BD00C78A24216D15A68016046
S1139F1042601A890281002A01D00136F6B25989B9
S1139F2041819A8982819B7BC373002901D1002AD4
S1139F3001D00137FFB2143001E01033E0E7019B98
S1139F4001330193D7E7026008E001340022A256EE
S1139F50002AFAD10134B7E7371C351C2C4C23688E
S1139F60002B49D0002F2CD00C207843043080B231
S1139F70FFF748FF274A2368106094461A68002AAE
S1139F801AD05A89002A07D024498A4201D10022D2
S1139F905A815A89426003E09989002901D04160BD
S1139FA001224168002901D001214172002A01D017
S1139FB003600C301433E1E70C235F436346C01B9A
S1139FC0186003997018C0B2FFF782FB002E13D0FB
S1139FD024682268002A0FD02389002B0AD003208A
S1139FE00121221CFFF722FC002801D0A07301E00C
S1139FF0FF23A3731434ECE7094801F085F9094BF6
S113A00000221A6001F04AFA281C05B0F0BDC046CF
S113A010BCFDFF1FC8FDFF1FD2FCFF1FFFFF000098
S113A020C0FDFF1FC4FDFF1F054A06481188CB076A
S113A030DB17034049084B4098B210807047C04674
S113A040C0FDFF1F00B4FFFF184B37B51C68236821
S113A050002B29D0E27B0D231A4223D001F064F9AE
S113A060A389002B02D1E37BD90716D4237C002BD0
S113A0700ED000256A46157055702168281C0A7890
S113A08069468A700522CD700B71FFF719FE25749D
S113A090E27B0A23134000D1E37301F04DF9201C45
S113A0A0626890471434D2E737BDC046BCFDFF1F39
S113A0B038B50C4B051C1C6801F036F92368002BDD
S113A0C00DD0E17B0D22114207D01B785BB2AB426D
S113A0D003D001F031F9012002E01434EEE7181C3A
S113A0E038BDC046BCFDFF1F074B1B681A68002A19
S113A0F007D0127852B2824201D1D87B02E01433E5
S113A100F4E780207047C046BCFDFF1F38B5174BED
S113A1101C682368002B27D01B785BB2834221D1B3
S113A120002918D1124B1D68002D14D02B68002B68
S113A13011D09C420DD101F0F7F8A389002B03D074
S113A1400C4A12689B186B600023E37301F0F4F867
S113A1500AE00C35EAE74A0702D5E37B1A0703D481
S113A160E17301E01434D4E738BDC046BCFDFF1FE1
S113A170C8FDFF1FC4FDFF1FF8B5194B0E1C1C685A
S113A180171C002C2BD0174B1D682B68002B26D0D6
S113A1901B785BB2834220D12368002B1FD09D42E1
S113A1A019D101F0C1F8EB7B02229343EB732772C0
S113A1B0002F04D1AE81002E04D1667208E0002E77
S113A1C000D10126084B1B68F618012366606372F0
S113A1D001F0B2F803E00C34DEE71435D5E7F8BD3E
S113A1E0C8FDFF1FBCFDFF1FC4FDFF1F38B5114B89
S113A1F01D68002D1DD0104B1C682368002B18D03F
S113A2001B785BB2834212D12B68002B11D09C4285
S113A2100BD101F089F800232B726B72E37B0222CD
S113A2201343E37301F088F803E00C35ECE71434CE
S113A230E3E738BDC8FDFF1FBCFDFF1F134A144BE5
S113A24011681B68013110B5101C1160002B1CD063
S113A2501A68002A19D0597A002914D001685C6858
S113A260A14210D1D17B8C0705D40C0701D4042161
S113A270D173197A11749289002A03D059688A1803
S113A2805A6000E05A720C33E2E710BDC4FDFF1FB0
S113A290C8FDFF1FF0B50D1C2C352B7885B0061CAE
S113A2A00C1C9A070FD01121DA0700D4132101F0F6
S113A2B033F9C0B2002861D12B78032293434022A2
S113A2C013432B705AE020271F4054D1088B0028D9
S113A2D003D1402293432B704DE0CA681178A26ADF
S113A2E0520516D50422134202D093432B7010E07A
S113A2F0221C2E3212780192914205D02D22125D39
S113A3008A4206D1012804D004210B4301992B7001
S113A3100127301C01F000F9236840220133236037
S113A3202B7813432B70002F28D1E3686269013323
S113A330E360934201D3A368E360228B104B013A9C
S113A340B600F35892B222832F34998C2378002BD1
S113A35014D08A4212D86A46937201230025D3721C
S113A360DD23157255721373281C02A90522FFF709
S113A370A7FC257002E0301C01F0EAF805B0F0BD3E
S113A380D8FDFF1FF7B5019308AB071C0D1C141C67
S113A3901E7800F0C9FF01980238082800D9F7E0B8
S113A3A001F088FD054A713CCAF6F6F6A1001423B3
S113A3B07A4A5E4312689319E90401D5DE6800E025
S113A3C09E68002C28D0E20703D5381C01F0FAF867
S113A3D004E0A30702D5381C01F018F9610703D57E
S113A3E0381C01F0C1F804E0220702D5381C01F042
S113A3F0DFF8B36AE10603D580225201134303E078
S113A400A20602D5664A1340B362630604D57F23CD
S113A4101D40331C2F331D70358DBAE01422564372
S113A4205E4B604A1B689E19B3689C6A144201D053
S113A4301D8CAEE01D8BACE01422584B56431B68B8
S113A4409E19F668002D07D1F28B338BD31A9DB277
S113A450A34200DB9DE09BE000F06EFF301C291C52
S113A460221C0830FFF772FB051C00F05DFF331C53
S113A4702C331A7860231A4200D08AE0381C311C2D
S113A480FFF708FF85E014237343444901930968E7
S113A490221CCB189E68291C301C0830FFF7E7FAF1
S113A4A0B36A6022051C134275D0321C2C32117819
S113A4B0102001426FD0348BA446B48CA4456AD8D2
S113A4C081431170990666D5344C01202668019C9D
S113A4D03619F1680B1C2C331A7802431A70381C95
S113A4E0FFF7D8FE57E02D4A1423012C08D95E4308
S113A4F01368023C9E19F368A4B2002D13D106E040
S113A5005E4312689619B368002D0CD107E0012C44
S113A51005D91D605D60B3681D605D6039E0A4000D
S113A5200025E55035E0A4001C190023E25CEA5440
S113A5300133042BFAD12BE0184D1423002C04D042
S113A5405E432A689619F3681BE05E432968102469
S113A5508A199368191C2C310878204211D0A04321
S113A5600870D1688A6A920608D50B1C2C331A78B5
S113A570012002431A70381CFFF78CFE2B689E19C9
S113A580B3689A6800251A61DA601D831D8400E0AF
S113A590002500F0D1FE281CFEBDC046ACFDFF1F07
S113A5A0FFEFFFFF8080000038B5051C3020FFF767
S113A5B029FC041E01D100200BE0281CFFF722FC1B
S113A5C0A0600028F7D043192061E0606361E5834F
S113A5D0201C38BDF7B53E4E0091017A041C301C96
S113A5E0FFF7BEF8051C071C002D03D0009A520784
S113A5F007D46BE0291CFFF7B3F8051C381C002DA9
S113A60064D014276F43334B143F1B68DF19009B3E
S113A6107E609B0707D5E088267AFFF7C5FF2E4AA0
S113A620B6009051F860009B2C4EDB0706D5A0883D
S113A630FFF7BAFF237AB8609B00F050237A264ACA
S113A6409B00D358002B0ED0226864219A62237A8F
S113A650214A9B00D358E0880093A37B584301F020
S113A6608BFC009B9884237A9B00F358002B26D004
S113A670227B2F331A70237AA288607B9B00F358C5
S113A680504364210092019301F076FC019B009AEF
S113A6905884237AA07B9B00F35850436421019390
S113A6A001F06AFC019B22689884237A9B00F3588A
S113A6B09A62237AA27A9B00F3582E331A70237A73
S113A6C0211C3B74207A00F0ABFF281CFEBDC04661
S113A6D085A30000ACFDFF1FD8FDFF1FCCFDFF1FAD
S113A6E0F7B55B4A8B009C585A4A80279D58A36A49
S113A6F03F01061C01911F4014D0221C2C321178FA
S113A70004200F1C0740BC4603D08143117000276E
S113A71010E0271C2E373F78B74202D10143117055
S113A72094E067461A0605D5221C2D321778BF1B04
S113A7307A4257412022134218D0132E08D12B1CE1
S113A7402C3319780A431A706B6801336B607DE00F
S113A750112E0BD12B1C2C331978114276D0914336
S113A76019700198291CFFF795FD6FE022680132EA
S113A7702260D9041AD52A8BEB8B9A420CD82A6909
S113A78016702B69696901332B618B4201D3AA6866
S113A7902A612B8B01332B832B1C2C331A786023D7
S113A7A01A4203D10198291CFFF774FD238BE28B15
S113A7B0002F32D19A420BD90133238323691E70AF
S113A7C02369676901332361BB4201D3A168216115
S113A7D0A36A602213421BD0261C2C363278D7067B
S113A7E016D4218B628C914212D3990609D52B1C65
S113A7F02C331A7802210A431A700198291CFFF796
S113A80049FD337810221343337063680133636066
S113A810114BA26A1A4211D018E0218C0131218413
S113A8209A420BD90133238323691E702369676914
S113A83001332361BB4201D3A16821612F34207805
S113A840002803D040B20421FFF760FCF7BDC046E6
S113A850CCFDFF1FD8FDFF1F8080000008B5034B0F
S113A8608200D158FFF716FD08BDC046D8FDFF1F72
S113A87070B5041C01200E1C151C00F085FF002877
S113A88007D100F081FF002800D141200323584064
S113A890C0B223B2002B05DA80235B421843C0B256
S113A8A0032358406404321C2B1C610C00F0B2FFDB
S113A8B070BD03B270B5041C0E1C151C0120002BC6
S113A8C002DA6404640C002000F05EFF002805D066
S113A8D0211C321C2B1C00F081FF01E001204042AE
S113A8E070BD08B5022804D003280ED0012817D162
S113A8F00CE0002000F048FF002811D080235B42C8
S113A90018430021C0B20A1C06E0002000F03CFFFE
S113A910002805D001210022131C00F07BFF01E078
S113A9200120404208BD08B500F0D8FD08BD000074
S113A9300B4B30B500221C1C00215956002908D0AD
S113A9405988814205D8002A02D055888D4200D901
S113A9501A1C211C06333C318B42EDD1101C30BD36
S113A960E6FDFF1F084B10B51C1C00229A56002A56
S113A97004D0834202D05A88521A5A80221C0633C9
S113A9803C329342F1D110BDE6FDFF1FF0B5807B50
S113A99089B00190019802A90522FEF7BFFE0028A4
S113A9A037D06B46DE7A002EF4D104AD1A4F2E70E8
S113A9B06E70EE70381CFFF7BBFF041E13D0174BEC
S113A9C067881B88BB4202D206AE73800DE02378F1
S113A9D00020AB702379291C2B7105222070FFF70E
S113A9E06FF9261CE6E7002E05D07188002902D0F5
S113A9F0301CFFF7B7FF0848FFF79AFF041EC9D0C1
S113AA00418801227020FFF7B7FB6288034B1A804C
S113AA10C0E709B0F0BDC046FFFF0000E4FDFF1F22
S113AA2008B56120B721FFF787F908BDF8B53D4B9C
S113AA303D4E1A68041C01321A6033780D1C013330
S113AA40DBB233703B2B4DD9384F3B780133DBB24B
S113AA503B703B2B39D9364B1A780132D2B2172AC4
S113AA6001D81A7024E000221A70324A3248117850
S113AA7003780131C9B211700133DBB2062B01D95D
S113AA80073BFAE703701D2907D12C4B19780229DB
S113AA9003D10121117003221A702A0708D5E36833
S113AAA0002B05D000F040FCE268904700F044FC25
S113AAB0AB0608D56269002A05D000F035FC63694D
S113AAC0984700F039FC00233B70AA0708D5636857
S113AAD0002B05D000F028FC6268904700F02CFCA5
S113AAE000233370EB0508D5A268002A05D000F0D6
S113AAF01BFCA368984700F01FFCAA0508D523682F
S113AB00002B05D000F010FC2268904700F014FCE4
S113AB102369002B05D000F007FC2369984700F057
S113AB200BFCF8BD24FEFF1F29FEFF1F2AFEFF1F9A
S113AB3028FEFF1FCEFCFF1FCDFCFF1FCFFCFF1F15
S113AB400D4B1B78C3720D4B1B8883800C4B1B78F9
S113AB5083710C4B1B78C3710B4B1B7803720B4B2B
S113AB601B7843720A4B1B7883720A4B1B68036180
S113AB70802303737047C04629FEFF1FD0FCFF1FCC
S113AB80CFFCFF1FCEFCFF1FCDFCFF1F28FEFF1FC5
S113AB902AFEFF1F24FEFF1FF0B58C46002801D1BA
S113ABA0414B1960414C62460423611E89B28D07F2
S113ABB00DD13F4DAA420FD93E4E02339219DBB25A
S113ABC0062B02D80134A4B2EFE7073BF7E73A4D6E
S113ABD0AA4204D8002500E00125002408E03749F2
S113ABE001335218DBB2062BECD9073BFAE70224F7
S113ABF0002D0CD0012C0AD1314EB24217D9314C60
S113AC001D331219DBB2062BF1D9073BFAE72E4E9E
S113AC102E4F365D7743BA4209D9D21BF318DBB203
S113AC20062B01D9073BFAE70134E4B2E0E701342B
S113AC30E4B20127254DAA4209D9254D01375219FD
S113AC40FFB20133DBB2062BF4D9073BFAE7002548
S113AC50204EB24204D9204E01359219EDB2F7E7E5
S113AC6000263B2A03D901363C3AF6B2F9E7D2B2C0
S113AC70002809D0818061468471C7710372C27251
S113AC808672457201610DE014480470144807701F
S113AC9014480370144B1A70144B1E70144B1D701F
S113ACA0144B1980F0BDC04624FEFF1FB3070000FB
S113ACB00085E201007B1DFE8033E10180CC1EFE95
S113ACC0803B260080C4D9FF62D00000805101007F
S113ACD080AEFEFF0F0E0000F0F1FFFFCFFCFF1F60
S113ACE0CEFCFF1FCDFCFF1F29FEFF1F2AFEFF1F06
S113ACF028FEFF1FD0FCFF1FF0B58BB005AD0190FF
S113AD000C1C281C00211422FEF7A0FE0199042922
S113AD1010D10B232B73002C0FD0281C00F0EEFD58
S113AD202A69002A09D1201C7949FFF72FF8001B52
S113AD30C0B2EAE0281CFFF703FF019B07261E4070
S113AD403AD0002C34D006261E40221C002E12D0ED
S113AD500021E879FEF784FD2E270770421C40216C
S113AD60A879FEF77DFD021C07700132A888002136
S113AD70FEF776FD021C01990523194219D0002E15
S113AD8002D02023137001324021687AFEF768FD57
S113AD903A260670421C4021A87AFEF761FD021C87
S113ADA006700132E87A4021FEF75AFD021C00E0E9
S113ADB0221C141BE0B2A8E0002C00D196E0019AFA
S113ADC0102A0AD10023E3562B2B0BD10134002384
S113ADD0E356202BFAD0012604E0019B302B01D14D
S113ADE010210191201CFEF70EFEC2B2071C039233
S113ADF023781A1C303A092A01D80134F8E70021D3
S113AE0002918B420FD00134201CFEF7FCFDC0B22E
S113AE1002902378303B092B01D80134F9E7331C25
S113AE205A1E9341F6180022A25600239A4208D0D3
S113AE300134201CFEF7E7FD321C511E8A4183B207
S113AE40B618019A102A10D12278111C3039092918
S113AE5001D80134F8E7211C202A06D14A780134AC
S113AE60303A092A01D830210191019A92060BD572
S113AE70029A0399AA71274AE971934202D8FA21E6
S113AE80C9005B18AB802DE0032E25D8301C01F0DF
S113AE9011F802080C15039A02996A72A972EB72EE
S113AEA020E02A69FFB2BF1806E03C23FFB25F43EB
S113AEB02B690299FF187F182F610FE0E12212011C
S113AEC0FFB257432A690299BF183C224A43DBB2B6
S113AED0BF18FB182B6101E0002E03D0281C296940
S113AEE0FFF75AFE019A302A00D179E7019B102B13
S113AEF004D1094B059306232B7302E0012205AB11
S113AF001A73281C00F0FAFC00200BB0F0BDC046F8
S113AF106ED00000CF07000021AA0000F0B587B072
S113AF20059181880422039135490023039C03265B
S113AF30A14214D24C1C314207D1324D02325B196A
S113AF40D2B2062A09D9073AFAE72F4F0132DB19A0
S113AF50D2B2062A01D9073AFAE7211CE6E70E40E5
S113AF6081794C1E002C0BD0284D013C655D284F87
S113AF70AA186F43DB19D2B2062AF3D9073AFAE7C3
S113AF80002E09D1022907D9214D01325B19D2B211
S113AF90062A01D9073AFAE7C679771ED219D2B23E
S113AFA0062A01D9073AFAE7447A0194857A049586
S113AFB0C47A019DE12000014543AC46049D3C2038
S113AFC0684302906044051911484743EF19F81883
S113AFD0059B002B12D00F4B039D019F1D800E4B30
S113AFE019700E4B04991E700D4B1F700D4B197088
S113AFF00D4B1C700D4B1A700D4B186007B0F0BD53
S113B000B20700000085E2018033E10162D0000054
S113B01080510100D0FCFF1FCFFCFF1FCEFCFF1F9F
S113B02028FEFF1F2AFEFF1F29FEFF1FCDFCFF1F66
S113B03024FEFF1F10B586B0041C422301A803732D
S113B040019400F05BFC021E012A05D1034B6B2026
S113B05014211C60FFF790F806B010BD2CFEFF1FF2
S113B06010B5847B88B0201C69460522FEF756FB88
S113B07000280BD06A46D378002BF4D11379012B26
S113B080F1D1034B1868FFF7D5FFECE708B010BD0A
S113B0902CFEFF1FF8B5204B051C1421186800F086
S113B0A01DFF1E49071C00F019FF2A1C0021041C67
S113B0B0FEF7D6FB194D44216C4341706121817028
S113B0C07921C17073213D1B20220171E12102709D
S113B0D0861D42710901281C00F000FF321C00216A
S113B0E0041CFEF7BDFBE1231B015C433A262C1B29
S113B0F0471C06703C21201C00F0F0FE3A1C402145
S113B100051CFEF7ADFB0670421C3C204543402164
S113B110601BFEF7A5FBF8BDC4FDFF1F80510100B5
S113B12008B56C20FEF7C4FF002801D100F0E0FC54
S113B13008BD704770477047704770477047704745
S113B1407047704770B5164C164D23782A78DBB2D9
S113B1501A4091060CD5144A144E90783378022183
S113B1601840FFF7BDFA2378DBB21A0700D532780E
S113B1702A783F218A431A4202D00220FFF76EFB4D
S113B1802A7840231A420AD02178194207D09A43D8
S113B190044B1A70064B042219689143196070BD60
S113B1A004C0064003C00640A8FEFF1F07C00640B7
S113B1B068FEFF1F70B5164C164D23782A78DBB253
S113B1C01A4091060CD5144A144E50783378012154
S113B1D01840FFF785FA2378DBB21A0700D53278D6
S113B1E02A783F218A431A4202D00120FFF736FB16
S113B1F02A7840231A420AD02178194207D09A4368
S113B200044B1A70064B022219689143196070BDF1
S113B21004B0064003B00640A8FEFF1F07B0064076
S113B22068FEFF1F70B5164C164D23782A78DBB2E2
S113B2301A4091060CD5144A144E10783378002124
S113B2401840FFF74DFA2378DBB21A0700D532789D
S113B2502A783F218A431A4202D00020FFF7FEFADF
S113B2602A7840231A420AD02178194207D09A43F7
S113B270044B1A70064B012219689143196070BD82
S113B28004A0064003A00640A8FEFF1F07A0064036
S113B29068FEFF1F154B10B51A68802001321A6032
S113B2A0134B144C1968014319602368590706D5D8
S113B2B0114909688A4202D14200134323600F4AAC
S113B2C01368002B08D0013B1360002B04D12268C3
S113B2D080239B001343236021680948FFF7A6FBE2
S113B2E02168084B0B40236010BDC046F80B0020BA
S113B2F000D0034064FEFF1F5CFEFF1F34FEFF1FEF
S113B3003CFEFF1FFFFCFFFF054B10B51C682388A4
S113B310002B00D1034B0380FEF786FE208010BD76
S113B320ACFEFF1F7B12000072B6024B1A6801329A
S113B3301A60704760FEFF1F034A1368013B1360E5
S113B340002B00D162B6704760FEFF1F08B5802253
S113B350044B92041A60FFF7E7FFFEF76FFFFFF755
S113B360EBFF08BD04ED00E0314BF7B51C68002C81
S113B37014D1304C01239C43251C3C35231C0195DE
S113B3802D4D1E882F1BDE53019F0233BB42F7D184
S113B390274C0135294B256013241C70284C237835
S113B3A05BB2002BFADA257830231D4200D02370DB
S113B3B0244D00232B70244B18709C46062801D082
S113B3C00A2827D10E0C214BF6B201271E702F70CC
S113B3D00F0AFFB26446C9B227701A4E1A4D19708B
S113B3E0062817D10221317051782970117819700B
S113B3F003213170D178297091781970042131704A
S113B400517929701179197005213170D179297018
S113B41092791A70FFF788FF054D094E2B6808488A
S113B4209847FFF789FF307833231840FEBDC046A4
S113B43038FEFF1FD4FCFF1F6CFEFF1F03000240F9
S113B44005000240010002400900024008000240D9
S113B4500E4B10B51B6884004033E2500C4A89013E
S113B4608318C9B21970C317DB0E1B18094A5B1184
S113B4709B009B18084A104004D5202201385242F0
S113B48010430130012282401A6010BD08ED00E033
S113B49000E400E000E100E01F000080084A094BDE
S113B4A0DA63094B094A1360094A1360094BC02245
S113B4B0196812060A431A60074B07221A6070477C
S113B4C04DB3000000FCFF1F7F841E0014E000E069
S113B4D018E000E020ED00E010E000E008B5094BC2
S113B4E01B785BB2002B08DAFFF71EFF064B074AF6
S113B4F01A80074A1A80FFF71FFF8022054B920427
S113B5001A6008BD0020054002200540A602000084
S113B510B480FFFF4C0000F810B50B4B8200D358E9
S113B52001221C7964B2002C0CDA084C8240206899
S113B530024322601A79D9718022D97852420A438F
S113B540DA700022101C10BD74D1000068FEFF1FC9
S113B550044B8000C3587F22D9780A4040210A4313
S113B560DA70704774D100000D4B820010B5011CD5
S113B570D45801280AD0002804D002280BD10E2068
S113B580084A06E00C200221074A02E0074A0D207F
S113B5900221FFF75DFFE37808221343E37010BD37
S113B5A074D1000045B1000025B20000B5B100001F
S113B5B0034B8000C3583722D9780A40DA707047A9
S113B5C074D100000D4B820010B5011CD458012821
S113B5D00AD0002804D002280BD10E20084A06E025
S113B5E00C200221074A02E0074A0D200221FFF73E
S113B5F02FFFE37824221343E37010BD74D10000BD
S113B60045B1000025B20000B5B10000034B800035
S113B610C3582421DA788A43DA70704774D1000061
S113B6201F4B820030B5D35801280BD0002805D019
S113B630022834D180241B4AE40306E08024194AFA
S113B640640302E08024174AA40315682C431460A1
S113B650CC7A41220B2C02D8134A6400A25AD40497
S113B660E40ED2B21C705A700A68104C0621D50739
S113B67009D57F252554114010D0510701D5032247
S113B6800AE0022208E0FF252554114006D05407A1
S113B69001D5132200E012229A7000E0997030BDA7
S113B6A074D100001480044080D00000A8FEFF1F65
S113B6B038B5440A451864020A20211C0022FFF709
S113B6C053FE002806D180232A1B9B009A4202D9EC
S113B6D0E418F1E7012038BD08B58021C900FFF75F
S113B6E0E7FF08BDF7B507230191161C204C00297C
S113B6F009D122681A4201D1002038E09A4322601D
S113B7000822009204E0021C9A4318402260009030
S113B710009B0825ED1AB54200D9351C154A009B3B
S113B7200199D718381C2A1CFEF798F9019A114B75
S113B73052197F1908330192761B9F4210D30620B9
S113B74021680C4AFFF710FE051E0FD12368094833
S113B7500833FF2108222360FEF778F9009502E000
S113B76023685D192560002ED2D1C5E70120FEBDF6
S113B77030FEFF1F54FEFF1F08B5031C081C191CD4
S113B780FEF76CF908BD000030B5F02185B0051C4A
S113B7900902684610226B425D41FEF75FF90E4CC8
S113B7A0009B6D422543A34202D1029BAB420FD0C2
S113B7B0F421684609021022FEF750F9009B00208C
S113B7C0A34206D10298401B45426841400000E074
S113B7D0012005B030BDC04655555555F8B5151C6A
S113B7E01E1C022801D0F02400E0F42424021034AA
S113B7F0C9000C19281CAA1992B283B29A4207D024
S113B800471C211C0122FEF729F90834381CF2E7F1
S113B8100020F8BDF0B585B00193002543B20F1C9C
S113B8200092AB4202DA7F2318400125410608D575
S113B830F0200002FFF750FFF4200002FFF74CFF56
S113B84002E0F424022800D0F024019B2402002BFF
S113B85011D1002D09D0F0200002844201D1F4203E
S113B8600002FFF739FF002520E0201CFFF734FF1A
S113B870002F1BD03BE0231C1033FF00FF180123D3
S113B8805B42009E0393019B0099CA1892B2B3B223
S113B8909A420BD03378174A381C134302A9082262
S113B8A002930837FFF71EFF0136ECE7211C02A8BC
S113B8B00822FEF7D3F8104E0299B14205D0201C9D
S113B8C002A908220296FFF70DFF002D0FD10834BC
S113B8D002A8211C0822FEF7C1F8029BB34206D03D
S113B8E0054B201C02A908220293FFF7FBFE00204F
S113B8F005B0F0BD00FFFFFF55555555F8B5037B66
S113B900041CF022181C904301380A2800D992E044
S113B91000F0D0FA08063E2A2D30831B1F2518009C
S113B920002522E0454D980606D521690020FFF741
S113B93033F924692C607EE0201C0121FFF7EEFA24
S113B940286078E03E4B19680AE0201CFFF7F8F8FD
S113B95071E0201C0021FFF7E1FA20616BE021690E
S113B960201CFFF719F966E00125013500E00025E8
S113B97001350BE0334A0421106820258843106008
S113B9801D402F4E43D0216900253160013500E070
S113B99000250135237B01272A4E7F2B04D93368E8
S113B9A0AF40BB43336046E0274B20681A6803214D
S113B9B03A431A60254BAA00D050254A1420FFF7B9
S113B9C047FD244B03211A78AF400A431A70224BD7
S113B9D09222920031681A603D1C204B204A0D438C
S113B9E01A603560237B5A0625D51E491E4B0888EC
S113B9F0124A984208D0002313601C4A13801C4A40
S113BA0013601C4B0B8016E011680020A9E7201C72
S113BA10291CFFF783FA3060B8E7637AE122120148
S113BA205A43A37A3C214B43D218E37A0025D21817
S113BA30114B1A60AEE70020F8BDC046F80B002099
S113BA405CFEFF1F64FEFF1F148004403CFEFF1FCA
S113BA5095B200000040064004D0034000D00340EB
S113BA60C0870000F20B002035CA0000F00B002054
S113BA70F40B002035CAFFFF34FEFF1F30B51A4C0B
S113BA8083001B191C68D50701D50C4300E08C43C7
S113BA901C6080240123640400280DD1080B03409A
S113BAA0880401D502200343214201D0042003432A
S113BAB08C010FD508210CE00B401B018D0701D52B
S113BAC020200343214201D040200343880101D5B3
S113BAD080210B430549940702D50D682B4301E0EF
S113BAE0086803400B6030BD089004401490044083
S113BAF0F8B5314B04211C68304A0C423FD0304821
S113BB000068002803D018688843011C36E01068D8
S113BB10C0020ED52B4840260578354305702A4DC2
S113BB202F783E432E700078C50702D518688843E5
S113BB301860106880020FD52449402508782843EE
S113BB40087023480678354305700978CD0703D576
S113BB501968042081431960106840020FD51D49FB
S113BB6040250878284308701B480678354305703B
S113BB700978CD0703D5196804208143196030BFC3
S113BB801C601068C00204D50F4B40201978814313
S113BB9019701168890204D50D4B4020197881432E
S113BBA0197013685A0204D50B4B40211A788A4342
S113BBB01A70FFF7C1FBF8BD10ED00E014800440DB
S113BBC068FEFF1F05A0064000A0064005B0064021
S113BBD000B0064005C0064000C0064008B56C2011
S113BBE0FEF782FA0923021C00201A4207D0044BF4
S113BBF0186804230340584243410220C01A08BD78
S113BC0010ED00E010B5E023041C9C43012C07D088
S113BC10022C0DD0002C10D16C20211CFEF776FADA
S113BC20084B04211A688A431A60002C05D108E0E5
S113BC30044B04211A680A431A606C200121FEF7A0
S113BC4065FA10BD10ED00E0014A024B1A60FEE7F0
S113BC500400FA050CED00E010B5124A1249002365
S113BC60891A8B4204D01148C05CD0540133F8E7E0
S113BC700F49104A914204D10F4A10490023891AEE
S113BC8008E00F480023801A8342F5D0CC5CD454DA
S113BC900133F9E78B4204D0D01800240470013337
S113BCA0F8E710BDC0FCFF1FE0FCFF1F80D10000BF
S113BCB01080000010800000E0FCFF1FB0FEFF1F9A
S113BCC03CC00000F8B5504D30212B684F4C8B43DD
S113BCD02B60236801208B43021C2360FFF7CEFEF8
S113BCE04B4B20201B684B4F03409C464A4E4B4B0A
S113BCF02A1C65461F804A491E80002D0BD1494EDF
S113BD00412333704848494B65460380484B1D80A6
S113BD1080230B7009E0434E002333700125424E0B
S113BD206D423580424D2B8008701168414B80254F
S113BD300B401360404BAD041A68291C2A431A6057
S113BD4001200222FFF79AFE23680C221D433B4B7D
S113BD5025601A603A4BB4221A701A78D607FCD5BB
S113BD60384B18221A70384B1A78191CD006FAD49A
S113BD700A78354B5506FBD5344A802149041160B5
S113BD80334A00211170197880220A431A70314B0A
S113BD90314A9A60314ADA60314A1A61314A5A6149
S113BDA0314A9A61314A1A63314A9A63314ADA62F2
S113BDB0314A3249116032498A4201D00432F8E7EB
S113BDC0304A1360FFF748FFFF2108222E48FDF791
S113BDD03DFE2E4B2E4A13602E4A13602E4B1A68DA
S113BDE005221A60FCF7BAFA2C4A2D4B2D482E492D
S113BDF01A60FDF7E1FF2D482D490322FEF758F89C
S113BE00FEF722F9FCE7C04658F00F4054F00F400B
S113BE1050F00F40C5200000D92800000220054042
S113BE2000200540012005400420054007D0FFFF05
S113BE3006200540FFFFFFFD40F00F400480044052
S113BE400050064000400640044006402480044060
S113BE500140064000FCFF1F41B1000033B1000067
S113BE6035B1000037B1000039B100003BB100002A
S113BE703DB100003FB1000040FCFF1F43B1000092
S113BE80B0FCFF1F08ED00E054FEFF1FFFFFFF00A2
S113BE9014E000E018E000E010E000E0FC0B0020FB
S113BEA0ACFEFF1F98D00000B0FEFF1FF8D00000CA
S113BEB068D1000002B4714649084900095C490090
S113BEC08E4402BC7047C04603B471464908400022
S113BED04900095A49008E4403BC7047002934D0F4
S113BEE00123002210B488422CD301242407A14248
S113BEF004D2814202D209011B01F8E7E400A14205
S113BF0004D2814202D249005B00F8E7884201D39F
S113BF10401A1A434C08A04202D3001B5C08224377
S113BF208C08A04202D3001B9C082243CC08A042E8
S113BF3002D3001BDC082243002803D01B0901D0D4
S113BF400909E3E7101C10BC7047002801D0002049
S113BF50C04307B4024802A14018029003BDC04682
S113BF60D90000000029F0D003B5FFF7B9FF0EBCDB
S113BF704243891A1847C046002941D010B4041C12
S113BF804C40A44601230022002900D54942002840
S113BF9000D5404288422CD301242407A14204D274
S113BFA0814202D209011B01F8E7E400A14204D254
S113BFB0814202D249005B00F8E7884201D3401A6B
S113BFC01A434C08A04202D3001B5C0822438C088D
S113BFD0A04202D3001B9C082243CC08A04202D3F7
S113BFE0001BDC082243002803D01B0901D00909E7
S113BFF0E3E7101C6446002C00D5404210BC704797
S113C000002806D003DB0020C043400801E0802064
S113C010000607B4024802A14018029003BDC046BE
S113C020190000000029EBD003B5FFF7A7FF0EBCF1
S10FC0304243891A1847C0467047C046B6
S113C03C210078002000000017005D600A00000059
S113C04C0041444D494E002020755461736B657258
S113C05C264B494E45544953000000000000000093
S113C06C0000000000005014030300000000000056
S113C07C0D0A0A48656C6C6F2C20776F726C642EF9
S113C08C2E2E204B494E455449530D0A004F532034
S113C09C4865617020757365203D20002066726FC1
S113C0AC6D200052544320416C61726D206669729C
S113C0BC65640D0A00436F6D6D616E64206C696E6E
S113C0CC6520626C6F636B65640D0A00436F6E6E62
S113C0DC656374696F6E2074696D6564206F757423
S113C0EC0D0A004C6F636B757000000005C70000EF
S113C0FC08C700000012000018C700001DC700008C
S113C10C02000000333030000000003630300000F4
S113C11C0000313230300000003234303000000086
S113C12C34383030000000393630300000003134FF
S113C13C3430300000313932303000003338343090
S113C14C3000003537363030000031313532303084
S113C15C003233303430300057444F470000000075
S113C16C05C7000008C700000012000018C7000033
S113C17C1DC700000200000005C7000008C700002E
S113C18C0012000046C7000030C700000000000089
S113C19C18C700001DC7000002000000536F66742E
S113C1AC776172650000000005C7000008C7000035
S113C1BC00120000D6CA0000DFCA0000050000000F
S113C1CCF4CA0000FDCA00000501000015CB0000F4
S113C1DC1ECB00000502000032CB00003ACB00005D
S113C1EC0503000055CB00005ECB000005040000E5
S113C1FC7ECB00008DCB000005150000A8CB000001
S113C20CB6CB0000051600007EC70000D3CB00009F
S113C21C051100009DC70000A2C700000306000022
S113C22C46C7000030C700000000000018C700001B
S113C23C1DC7000002000000436C6F636B206C6F21
S113C24C7373000005C7000008C70000001200004B
S113C25C18C700001DC7000002000000536F66746D
S113C26C776172652076657273696F6E20000A0AB5
S113C27C0D000A0D3D3D3D3D3D3D3D3D3D3D3D3DAE
S113C28C3D3D3D3D3D3D3D0A0D000A0D5365726932
S113C29C616C206E756D6265723A20004465766936
S113C2AC6365206964656E74696669636174696F3A
S113C2BC6E3A20004E657720616C61726D20736557
S113C2CC740D0A00416C61726D20636C656172655A
S113C2DC640D0A004E65772074696D65207365746E
S113C2EC0D0A004E65772064617465207365740DC6
S113C2FC0A0030203D2052554E0031203D2057413C
S113C30C49540032203D2053544F5000205B61634C
S113C31C746976655D004C61737420726573657421
S113C32C206361757365203D20000A0D5379737485
S113C33C656D206D656D6F7279207573653A0A0DA4
S113C34C00467265652068656170203D20000A0D09
S113C35C556E7573656420737461636B203D2000A6
S113C36C202800290A0D000D0A546865206465769E
S113C37C69636520686173206265656E206F706502
S113C38C726174696E6720666F722000426164206A
S113C39C706F7274206E756D6265720D0A000D0AF1
S113C3AC506F727420646972656374696F6E3A209D
S113C3BC004F55545055540D0A00494E5055540DC8
S113C3CC0A00496E76616C696420706F72740D0A90
S113C3DC00506F727420697320696E7075740D0A45
S113C3EC00506F72742073746174653A2000310DBF
S113C3FC0A00300D0A000D0A3F3F0D0A23004D655B
S113C40C6D6F727920446973706C61790D0A002028
S113C41C2020200046696C6C0D0A00577269746503
S113C42C0D0A004572617365640D0A0045726173EF
S113C43C65206661696C6564210D0A000A0D4279F8
S113C44C65204279650A0D000A0D506172616D65B3
S113C45C746572207365740A0D000A0D54656D7051
S113C46C2E20506172616D65746572207365740A57
S113C47C0D000A0D506172616D65746572207661F0
S113C48C6C7565203D20000A0D4E6F2076616C6939
S113C49C6420706172616D6574657273206176617C
S113C4AC696C61626C650A0D000A0D4F72696769EB
S113C4BC6E616C20706172616D657465727320724B
S113C4CC6573746F7265640A0D000A0D46616374BA
S113C4DC6F727920706172616D657465727320720C
S113C4EC6573746F7265640A0D000A0D5061726194
S113C4FC6D657465727320696E76616C69646174C0
S113C50C65640A0D000A0D4E657720506172616DE9
S113C51C65746572732076616C6964617465640A10
S113C52C0D000A0D436F6E66696775726174696FED
S113C53C6E2073617665640A0D00496E636F7272C6
S113C54C6563742064617461206C656E6774680D36
S113C55C0A000D0A53657269616C20636F6E66691B
S113C56C6775726174696F6E0D0A0042617564209F
S113C57C3D2000696E76616C6964210037003800D7
S113C58C20426974730D0A002073746F7020626901
S113C59C742873290D0A00466C6F7720636F6E74D0
S113C5AC726F6C200048696768207761746572202B
S113C5BC00250D0A004C6F7720776174657220009A
S113C5CC656E61626C650064697361626C65000D13
S113C5DC0A496E76616C6964207377697463680DBB
S113C5EC0A00496E636F72726563742073657269B5
S113C5FC616C2073706565640D0A00496E636F721B
S113C60C72656374207061726974790D0A00496EE5
S113C61C636F72726563742073746F7020626974D3
S113C62C730D0A00496E636F727265637420666CD5
S113C63C6F7720636F6E74726F6C0D0A000A0D0DA8
S113C64C004D41430020202020204D61696E206D57
S113C65C656E7500204C414E20636F6E666967757C
S113C66C726174696F6E0020202053657269616C6D
S113C67C20636F6E6669672E0020496E7075742F87
S113C68C4F7574707574206D656E75002020204193
S113C69C646D696E2E206D656E75002020205374B8
S113C6AC6174732E206D656E750020202020555307
S113C6BC42206D656E750020202020493243206D88
S113C6CC656E750020204469736B20696E74657205
S113C6DC66616365004654502F54454C4E455420B6
S113C6EC636F6D6D616E64730020202043414E2096
S113C6FC636F6D6D616E647300757000676F207489
S113C70C6F206D61696E206D656E7500717569744D
S113C71C004C6561766520636F6D6D616E64206D90
S113C72C6F646500446973706C6179206D656E7516
S113C73C2073706563696669632068656C70007545
S113C74C705F74696D650053686F77206F706572E4
S113C75C6174696E672074696D65006D656D6F72C7
S113C76C790053686F77206D656D6F7279207573DE
S113C77C650073686F775F636F6E666967005368F3
S113C78C6F7720636F6E66696775726174696F6E1B
S113C79C0073617665005361766520636F6E66691C
S113C7AC6775726174696F6E20746F20464C4153C7
S113C7BC480072656A656374005265736574206E13
S113C7CC6F6E2D7361766564206368616E67657343
S113C7DC00726573746F726500526573746F726561
S113C7EC20666163746F72792073657474696E6703
S113C7FC730073686F775F74696D65004469737057
S113C80C6C617920646174652F74696D650073655E
S113C81C745F74696D65005365742074696D65206B
S113C82C68683A6D6D3A7373007365745F64617410
S113C83C650053657420446174652064643A6D6DBD
S113C84C3A797979790073686F775F616C61726D8D
S113C85C00446973706C617920616C61726D206441
S113C86C2F74007365745F616C61726D0053657431
S113C87C20616C61726D20286461746529282B29F0
S113C88C5B74696D655D0064656C5F616C61726D90
S113C89C0044656C65746520616C61726D0073682D
S113C8AC6F775F6C700053686F77206C6F772070B4
S113C8BC6F776572206D6F646520616E64206F7094
S113C8CC74696F6E73007365745F6C70005B6F706A
S113C8DC74696F6E5D20536574206C6F7720706F74
S113C8EC776572206D6F64650072657365740052B0
S113C8FC6573657420646576696365006C61737433
S113C90C5F7273740052657365742063617573652B
S113C91C006D64004D656D6F727920446973706CA1
S113C92C6179205B616464726573735D205B3C6C3C
S113C93C3E7C3C773E7C3C623E5D205B6E756D5D5F
S113C94C006D6D004D656D6F7279204D6F64696675
S113C95C79205B616464726573735D205B3C6C3E2F
S113C96C7C3C773E7C3C623E5D205B76616C5D007A
S113C97C6D66004D656D6F72792046696C6C205B39
S113C98C616464726573735D205B3C6C3E7C3C77C4
S113C99C3E7C3C623E5D205B76616C5D205B6E751B
S113C9AC6D5D0073640053746F7261676520446934
S113C9BC73706C6179207B6173206D647D00736D81
S113C9CC0053746F72616765204D6F6469667920DA
S113C9DC7B6173206D6D7D0073660053746F72619F
S113C9EC67652046696C6C207B6173206D667D00E5
S113C9FC53746F72616765204572617365205B6166
S113CA0C6464726573735D205B6C656E2D68657808
S113CA1C5D007365745F6464720053657420706F99
S113CA2C72742074797065205B312E2E345D205B1A
S113CA3C3C693E7C3C6F3E006765745F64647200C5
S113CA4C47657420646174612064697265637469F8
S113CA5C6F6E205B312E2E345D00726561645F70E5
S113CA6C6F7274005265616420706F727420696E09
S113CA7C707574205B312E2E345D00777269746589
S113CA8C5F706F72740053657420706F7274206FD2
S113CA9C7574707574205B312E2E345D205B302FD1
S113CAAC315D0054656D7020746573740053617648
S113CABC6520706F72742073657474696E6720617D
S113CACC732064656661756C74007365745F626170
S113CADC7564005365742073657269616C206261BE
S113CAEC75642072617465007365745F73746F7020
S113CAFC005365742073746F7020626974732028FA
S113CB0C312F312E352F3229007365745F626974AD
S113CB1C73005365742064617461206269747320BA
S113CB2C28372F3829007365745F70617200536560
S113CB3C742070617269747920284556454E2F4FC4
S113CB4C44442F4E4F4E4529007365745F666C6FD9
S113CB5C770053657420666C6F7720636F6E747204
S113CB6C6F6C2028584F4E2F5254532F4E4F4E4516
S113CB7C29007365745F686967685F7761746572AF
S113CB8C0053657420666C6F77207374616C6C2031
S113CB9C282529205B312E2E39395D007365745F8D
S113CBAC6C6F775F77617465720053657420666C83
S113CBBC6F77207265737461727420282529205B49
S113CBCC312E2E39395D0053686F77207365726985
S113CBDC616C20636F6E66696775726174696F6EE0
S113CBEC003100436F6E666967757265204C414E67
S113CBFC20696E74657266616365003200436F6E02
S113CC0C6669677572652073657269616C20696EFB
S113CC1C74657266616365003300476F20746F201E
S113CC2C492F4F206D656E75003400476F20746F6B
S113CC3C2061646D696E697374726174696F6E20BE
S113CC4C6D656E75003500476F20746F206F7665C7
S113CC5C72766965772F737461746973746963731D
S113CC6C206D656E75003600476F20746F20555328
S113CC7C42206D656E7500476F20746F20493243F6
S113CC8C206D656E7500476F20746F207574464176
S113CC9C54206469736B20696E7465726661636594
S113CCAC0039004654502F54454C4E455420636C67
S113CCBC69656E7420636F6D6D616E6473006100E1
S113CCCC05C7000008C70000001200001DC90000C1
S113CCDC20C90000010F00004DC9000050C900001C
S113CCEC011000007CC900007FC900000111000084
S113CCFCAFC90000B2C9000001210000CAC900007C
S113CD0CCDC9000001220000E4C90000E7C90000FD
S113CD1C012300007BC70000FCC9000001250000B2
S113CD2C1ECA000026CA00000102000044CA00000A
S113CD3C4CCA0000010B000066CA000070CA000057
S113CD4C0104000087CA000092CA0000010500001B
S113CD5CB4CA0000AFCA0000014B00009DC700001C
S113CD6CB9CA0000010C000046C7000030C700001F
S113CD7C0000000018C700001DC7000002000000DE
S113CD8C7065726970686572616C206661696C7536
S113CD9C7265000074CF00000F0C000051C6000037
S113CDAC04D000001402000060C60000B4C10000EE
S113CDBC160C000073C60000CCCC00000F10000051
S113CDCC85C6000090CE00001111000098C600002A
S113CDDC44CE000011050000A7C6000084C1000069
S113CDEC0D030000B6C600005CCF00000D0200006D
S113CDFCC3C6000050C200000D020000D0C60000E3
S113CE0CF8C000000F020000E1C600006CC1000075
S113CE1C0F020000F5C60000486F7374206465624D
S113CE2C7567676572003F3F3F0031000000312E8B
S113CE3C350032000000000005C7000008C70000E0
S113CE4C001200004BC7000053C70000010A000089
S113CE5C67C700006EC700000101000046C7000050
S113CE6C30C700000000000018C700001DC70000F8
S113CE7C02000000556E646572766F6C74616765B0
S113CE8C0000000005C7000008C7000000120000E5
S113CE9C7EC700008AC70000060200009DC7000080
S113CEACA2C7000003060000BEC70000C5C70000EF
S113CEBC03070000DDC70000E5C700000302000003
S113CECCFEC7000008C80000060A00001AC80000CB
S113CEDC23C800000609000035C800003EC8000045
S113CEEC0608000052C800005DC80000060C0000D3
S113CEFC6FC8000079C80000060B000093C800003E
S113CF0C9DC80000060D0000AAC80000B2C80000AD
S113CF1C01260000D2C80000D9C800000127000077
S113CF2CF5C80000FBC800000100000008C900009F
S113CF3C11C900000120000046C7000030C70000E2
S113CF4C0000000018C700001DC70000020000000C
S113CF5C05C7000008C700000012000018C7000035
S113CF6C1DC7000002000000EDCB0000EFCB000059
S113CF7C0004000007CC000009CC000000050000F0
S113CF8C24CC000026CC00000006000035CC0000A8
S113CF9C37CC00000007000051CC000053CC00003B
S113CFAC0009000072CC000074CC0000000A0000E0
S113CFBC88C5000083CC0000000E00008AC5000068
S113CFCC92CC0000000F0000ADCC0000AFCC0000F0
S113CFDC00100000CACC0000F8C6000000110000CC
S113CFEC46C7000030C700000000000018C700004E
S113CFFC1DC700000200000005C7000008C70000A0
S113D00C0012000018C700001DC700000200000039
S113D01C4F444400004556454E004E4F4E45004586
S113D02C787465726E616C004E4F4E4500000000C2
S113D03C5254530000000000584F4E0000000000F2
S113D04C506F7765722D6F6E000820080056312ED4
S113D05C342E303132001F1C1F1E1F1E1F1F1E1F9B
S113D06C1E1F4E6F20616C61726D20656E61626C67
S113D07C65640000471023081204090204018200AD
S113D08C57004100210016000B00050001000008A8
S113D09C0000000048544D004A50470047494600E0
S113D0AC504E4700435353004A530042494E0054D8
S113D0BC58540049434F00424D50003F3F3F0057E6
S113D0CC646F670061707000706572696F64006DE5
S113D0DC61696E74656E616365006B65657065721C
S113D0EC006C6F77506F776572000000CBD0000036
S113D0FC27A900000000000004000100D0D00000AB
S113D10CD58100004500020000000000D4D00000CE
S113D11C8DA900002500FFFF00000000DBD00000FB
S113D12C058500002500FFFF00000000E6D000008C
S113D13C61B000002500FFFF00000000EDD00000EE
S113D14C21B10000000000000000010000000000FC
S113D15C0000000000000000000000000157616D99
S113D16C706B6C000000000000A0064000B006408C
S107D17C00C00640A5
S113D180FF0000000100000001000000FF04010195
S113D190B20701008021017001780906FCD57047AF
S90380106C
